
C:\Documents and Settings\jarek\Pulpit\Privet\Magisterka\Programy\1\um0427\FWLib\project\RIDE\STM3210E-EVAL\RTC.o:     file format elf32-littlearm
C:\Documents and Settings\jarek\Pulpit\Privet\Magisterka\Programy\1\um0427\FWLib\project\RIDE\STM3210E-EVAL\RTC.o

Disassembly of section .text.RTC_Init:

00000000 <RTC_Init>:
RTC_Init():
C:\Documents and Settings\jarek\Pulpit\Privet\Magisterka\Programy\1\um0427\FWLib\project/RTC.c:43
   0:	4770      	bx	lr
   2:	46c0      	nop			(mov r8, r8)
Disassembly of section .text.RTC_Thret:

00000000 <RTC_Thret>:
RTC_Thret():
C:\Documents and Settings\jarek\Pulpit\Privet\Magisterka\Programy\1\um0427\FWLib\project/RTC.c:48
   0:	480e      	ldr	r0, [pc, #56]	(3c <RTC_Thret+0x3c>)
C:\Documents and Settings\jarek\Pulpit\Privet\Magisterka\Programy\1\um0427\FWLib\project/RTC.c:49
   2:	f44f 727a 	mov.w	r2, #1000	; 0x3e8
C:\Documents and Settings\jarek\Pulpit\Privet\Magisterka\Programy\1\um0427\FWLib\project/RTC.c:48
   6:	6803      	ldr	r3, [r0, #0]
   8:	3301      	adds	r3, #1
C:\Documents and Settings\jarek\Pulpit\Privet\Magisterka\Programy\1\um0427\FWLib\project/RTC.c:49
   a:	fb93 f1f2 	sdiv	r1, r3, r2
   e:	fb01 3212 	mls	r2, r1, r2, r3
C:\Documents and Settings\jarek\Pulpit\Privet\Magisterka\Programy\1\um0427\FWLib\project/RTC.c:48
  12:	6003      	str	r3, [r0, #0]
C:\Documents and Settings\jarek\Pulpit\Privet\Magisterka\Programy\1\um0427\FWLib\project/RTC.c:49
  14:	b982      	cbnz	r2, 38 <RTC_Thret+0x38>
C:\Documents and Settings\jarek\Pulpit\Privet\Magisterka\Programy\1\um0427\FWLib\project/RTC.c:51
  16:	4a0a      	ldr	r2, [pc, #40]	(40 <RTC_Thret+0x40>)
C:\Documents and Settings\jarek\Pulpit\Privet\Magisterka\Programy\1\um0427\FWLib\project/RTC.c:50
  18:	2101      	movs	r1, #1
C:\Documents and Settings\jarek\Pulpit\Privet\Magisterka\Programy\1\um0427\FWLib\project/RTC.c:51
  1a:	6813      	ldr	r3, [r2, #0]
C:\Documents and Settings\jarek\Pulpit\Privet\Magisterka\Programy\1\um0427\FWLib\project/RTC.c:50
  1c:	6001      	str	r1, [r0, #0]
C:\Documents and Settings\jarek\Pulpit\Privet\Magisterka\Programy\1\um0427\FWLib\project/RTC.c:51
  1e:	185b      	adds	r3, r3, r1
  20:	6013      	str	r3, [r2, #0]
C:\Documents and Settings\jarek\Pulpit\Privet\Magisterka\Programy\1\um0427\FWLib\project/RTC.c:53
  22:	6843      	ldr	r3, [r0, #4]
  24:	b113      	cbz	r3, 2c <RTC_Thret+0x2c>
C:\Documents and Settings\jarek\Pulpit\Privet\Magisterka\Programy\1\um0427\FWLib\project/RTC.c:54
  26:	6853      	ldr	r3, [r2, #4]
  28:	185b      	adds	r3, r3, r1
  2a:	6053      	str	r3, [r2, #4]
C:\Documents and Settings\jarek\Pulpit\Privet\Magisterka\Programy\1\um0427\FWLib\project/RTC.c:56
  2c:	6883      	ldr	r3, [r0, #8]
  2e:	b113      	cbz	r3, 36 <RTC_Thret+0x36>
C:\Documents and Settings\jarek\Pulpit\Privet\Magisterka\Programy\1\um0427\FWLib\project/RTC.c:57
  30:	6893      	ldr	r3, [r2, #8]
  32:	3301      	adds	r3, #1
  34:	6093      	str	r3, [r2, #8]
C:\Documents and Settings\jarek\Pulpit\Privet\Magisterka\Programy\1\um0427\FWLib\project/RTC.c:59
  36:	60c1      	str	r1, [r0, #12]
C:\Documents and Settings\jarek\Pulpit\Privet\Magisterka\Programy\1\um0427\FWLib\project/RTC.c:61
  38:	4770      	bx	lr
  3a:	46c0      	nop			(mov r8, r8)
	...
Disassembly of section .text.RTC_Refresh:

00000000 <RTC_Refresh>:
RTC_Refresh():
C:\Documents and Settings\jarek\Pulpit\Privet\Magisterka\Programy\1\um0427\FWLib\project/RTC.c:65
   0:	4b01      	ldr	r3, [pc, #4]	(8 <RTC_Refresh+0x8>)
   2:	68d8      	ldr	r0, [r3, #12]
   4:	4770      	bx	lr
   6:	46c0      	nop			(mov r8, r8)
   8:	00000000 	.word	0x00000000
Disassembly of section .text.RTC_Pause:

00000000 <RTC_Pause>:
RTC_Pause():
C:\Documents and Settings\jarek\Pulpit\Privet\Magisterka\Programy\1\um0427\FWLib\project/RTC.c:68
   0:	2801      	cmp	r0, #1
   2:	d002      	beq.n	a <RTC_Pause+0xa>
   4:	2802      	cmp	r0, #2
   6:	d004      	beq.n	12 <RTC_Pause+0x12>
   8:	e006      	b.n	18 <RTC_Pause+0x18>
C:\Documents and Settings\jarek\Pulpit\Privet\Magisterka\Programy\1\um0427\FWLib\project/RTC.c:70
   a:	4b04      	ldr	r3, [pc, #16]	(1c <RTC_Pause+0x1c>)
   c:	2200      	movs	r2, #0
   e:	605a      	str	r2, [r3, #4]
C:\Documents and Settings\jarek\Pulpit\Privet\Magisterka\Programy\1\um0427\FWLib\project/RTC.c:71
  10:	e002      	b.n	18 <RTC_Pause+0x18>
C:\Documents and Settings\jarek\Pulpit\Privet\Magisterka\Programy\1\um0427\FWLib\project/RTC.c:73
  12:	4b02      	ldr	r3, [pc, #8]	(1c <RTC_Pause+0x1c>)
  14:	2200      	movs	r2, #0
  16:	609a      	str	r2, [r3, #8]
C:\Documents and Settings\jarek\Pulpit\Privet\Magisterka\Programy\1\um0427\FWLib\project/RTC.c:76
  18:	4770      	bx	lr
  1a:	46c0      	nop			(mov r8, r8)
  1c:	00000000 	.word	0x00000000
Disassembly of section .text.RTC_Play:

00000000 <RTC_Play>:
RTC_Play():
C:\Documents and Settings\jarek\Pulpit\Privet\Magisterka\Programy\1\um0427\FWLib\project/RTC.c:78
   0:	2801      	cmp	r0, #1
   2:	d002      	beq.n	a <RTC_Play+0xa>
   4:	2802      	cmp	r0, #2
   6:	d003      	beq.n	10 <RTC_Play+0x10>
   8:	e005      	b.n	16 <RTC_Play+0x16>
C:\Documents and Settings\jarek\Pulpit\Privet\Magisterka\Programy\1\um0427\FWLib\project/RTC.c:80
   a:	4b03      	ldr	r3, [pc, #12]	(18 <RTC_Play+0x18>)
   c:	6058      	str	r0, [r3, #4]
C:\Documents and Settings\jarek\Pulpit\Privet\Magisterka\Programy\1\um0427\FWLib\project/RTC.c:81
   e:	e002      	b.n	16 <RTC_Play+0x16>
C:\Documents and Settings\jarek\Pulpit\Privet\Magisterka\Programy\1\um0427\FWLib\project/RTC.c:83
  10:	4b01      	ldr	r3, [pc, #4]	(18 <RTC_Play+0x18>)
  12:	2201      	movs	r2, #1
  14:	609a      	str	r2, [r3, #8]
C:\Documents and Settings\jarek\Pulpit\Privet\Magisterka\Programy\1\um0427\FWLib\project/RTC.c:86
  16:	4770      	bx	lr
  18:	00000000 	.word	0x00000000
Disassembly of section .text.RTC_Validate:

00000000 <RTC_Validate>:
RTC_Validate():
C:\Documents and Settings\jarek\Pulpit\Privet\Magisterka\Programy\1\um0427\FWLib\project/RTC.c:230
   0:	6803      	ldr	r3, [r0, #0]
   2:	2b3b      	cmp	r3, #59
   4:	dd01      	ble.n	a <RTC_Validate+0xa>
C:\Documents and Settings\jarek\Pulpit\Privet\Magisterka\Programy\1\um0427\FWLib\project/RTC.c:231
   6:	233b      	movs	r3, #59
   8:	6003      	str	r3, [r0, #0]
C:\Documents and Settings\jarek\Pulpit\Privet\Magisterka\Programy\1\um0427\FWLib\project/RTC.c:234
   a:	6803      	ldr	r3, [r0, #0]
   c:	2b00      	cmp	r3, #0
   e:	da01      	bge.n	14 <RTC_Validate+0x14>
C:\Documents and Settings\jarek\Pulpit\Privet\Magisterka\Programy\1\um0427\FWLib\project/RTC.c:235
  10:	2300      	movs	r3, #0
  12:	6003      	str	r3, [r0, #0]
C:\Documents and Settings\jarek\Pulpit\Privet\Magisterka\Programy\1\um0427\FWLib\project/RTC.c:238
  14:	6843      	ldr	r3, [r0, #4]
  16:	2b3b      	cmp	r3, #59
  18:	dd01      	ble.n	1e <RTC_Validate+0x1e>
C:\Documents and Settings\jarek\Pulpit\Privet\Magisterka\Programy\1\um0427\FWLib\project/RTC.c:239
  1a:	233b      	movs	r3, #59
  1c:	6043      	str	r3, [r0, #4]
C:\Documents and Settings\jarek\Pulpit\Privet\Magisterka\Programy\1\um0427\FWLib\project/RTC.c:242
  1e:	6843      	ldr	r3, [r0, #4]
  20:	2b00      	cmp	r3, #0
  22:	da01      	bge.n	28 <RTC_Validate+0x28>
C:\Documents and Settings\jarek\Pulpit\Privet\Magisterka\Programy\1\um0427\FWLib\project/RTC.c:243
  24:	2300      	movs	r3, #0
  26:	6043      	str	r3, [r0, #4]
C:\Documents and Settings\jarek\Pulpit\Privet\Magisterka\Programy\1\um0427\FWLib\project/RTC.c:246
  28:	6883      	ldr	r3, [r0, #8]
  2a:	2b17      	cmp	r3, #23
  2c:	dd01      	ble.n	32 <RTC_Validate+0x32>
C:\Documents and Settings\jarek\Pulpit\Privet\Magisterka\Programy\1\um0427\FWLib\project/RTC.c:247
  2e:	2317      	movs	r3, #23
  30:	6083      	str	r3, [r0, #8]
C:\Documents and Settings\jarek\Pulpit\Privet\Magisterka\Programy\1\um0427\FWLib\project/RTC.c:250
  32:	6883      	ldr	r3, [r0, #8]
  34:	2b00      	cmp	r3, #0
  36:	da01      	bge.n	3c <RTC_Validate+0x3c>
C:\Documents and Settings\jarek\Pulpit\Privet\Magisterka\Programy\1\um0427\FWLib\project/RTC.c:251
  38:	2300      	movs	r3, #0
  3a:	6083      	str	r3, [r0, #8]
C:\Documents and Settings\jarek\Pulpit\Privet\Magisterka\Programy\1\um0427\FWLib\project/RTC.c:257
  3c:	68c3      	ldr	r3, [r0, #12]
  3e:	2b00      	cmp	r3, #0
  40:	da01      	bge.n	46 <RTC_Validate+0x46>
C:\Documents and Settings\jarek\Pulpit\Privet\Magisterka\Programy\1\um0427\FWLib\project/RTC.c:258
  42:	2300      	movs	r3, #0
  44:	6083      	str	r3, [r0, #8]
C:\Documents and Settings\jarek\Pulpit\Privet\Magisterka\Programy\1\um0427\FWLib\project/RTC.c:261
  46:	4770      	bx	lr
Disassembly of section .text.gday:

00000000 <gday>:
gday():
C:\Documents and Settings\jarek\Pulpit\Privet\Magisterka\Programy\1\um0427\FWLib\project/RTC.c:274
   0:	6903      	ldr	r3, [r0, #16]
   2:	210c      	movs	r1, #12
   4:	3309      	adds	r3, #9
   6:	fb93 f2f1 	sdiv	r2, r3, r1
   a:	fb02 3111 	mls	r1, r2, r1, r3
C:\Documents and Settings\jarek\Pulpit\Privet\Magisterka\Programy\1\um0427\FWLib\project/RTC.c:269
   e:	b510      	push	{r4, lr}
C:\Documents and Settings\jarek\Pulpit\Privet\Magisterka\Programy\1\um0427\FWLib\project/RTC.c:272
  10:	6944      	ldr	r4, [r0, #20]
C:\Documents and Settings\jarek\Pulpit\Privet\Magisterka\Programy\1\um0427\FWLib\project/RTC.c:275
  12:	220a      	movs	r2, #10
  14:	fb91 f3f2 	sdiv	r3, r1, r2
C:\Documents and Settings\jarek\Pulpit\Privet\Magisterka\Programy\1\um0427\FWLib\project/RTC.c:272
  18:	f5a4 64fa 	sub.w	r4, r4, #2000	; 0x7d0
C:\Documents and Settings\jarek\Pulpit\Privet\Magisterka\Programy\1\um0427\FWLib\project/RTC.c:275
  1c:	1ae4      	subs	r4, r4, r3
C:\Documents and Settings\jarek\Pulpit\Privet\Magisterka\Programy\1\um0427\FWLib\project/RTC.c:276
  1e:	68c3      	ldr	r3, [r0, #12]
  20:	f240 106d 	movw	r0, #365	; 0x16d
  24:	f5a3 7398 	sub.w	r3, r3, #304	; 0x130
  28:	3b03      	subs	r3, #3
  2a:	fb04 3000 	mla	r0, r4, r0, r3
  2e:	2304      	movs	r3, #4
  30:	fb94 f3f3 	sdiv	r3, r4, r3
  34:	18c0      	adds	r0, r0, r3
  36:	f44f 73c8 	mov.w	r3, #400	; 0x190
  3a:	fb94 f3f3 	sdiv	r3, r4, r3
  3e:	18c0      	adds	r0, r0, r3
  40:	f44f 7399 	mov.w	r3, #306	; 0x132
  44:	fb01 f103 	mul.w	r1, r1, r3
  48:	3105      	adds	r1, #5
  4a:	fb91 f1f2 	sdiv	r1, r1, r2
  4e:	2364      	movs	r3, #100
  50:	1840      	adds	r0, r0, r1
  52:	fb94 f4f3 	sdiv	r4, r4, r3
C:\Documents and Settings\jarek\Pulpit\Privet\Magisterka\Programy\1\um0427\FWLib\project/RTC.c:279
  56:	1b00      	subs	r0, r0, r4
  58:	bd10      	pop	{r4, pc}
  5a:	46c0      	nop			(mov r8, r8)
Disassembly of section .text.dtf:

00000000 <dtf>:
dtf():
C:\Documents and Settings\jarek\Pulpit\Privet\Magisterka\Programy\1\um0427\FWLib\project/RTC.c:283
   0:	f500 7099 	add.w	r0, r0, #306	; 0x132
C:\Documents and Settings\jarek\Pulpit\Privet\Magisterka\Programy\1\um0427\FWLib\project/RTC.c:284
   4:	f242 7310 	movw	r3, #10000	; 0x2710
   8:	fb00 f303 	mul.w	r3, r0, r3
   c:	4a25      	ldr	r2, [pc, #148]	(a4 <dtf+0xa4>)
   e:	f503 5366 	add.w	r3, r3, #14720	; 0x3980
  12:	333c      	adds	r3, #60
C:\Documents and Settings\jarek\Pulpit\Privet\Magisterka\Programy\1\um0427\FWLib\project/RTC.c:281
  14:	b5f0      	push	{r4, r5, r6, r7, lr}
C:\Documents and Settings\jarek\Pulpit\Privet\Magisterka\Programy\1\um0427\FWLib\project/RTC.c:285
  16:	2704      	movs	r7, #4
C:\Documents and Settings\jarek\Pulpit\Privet\Magisterka\Programy\1\um0427\FWLib\project/RTC.c:281
  18:	460d      	mov	r5, r1
C:\Documents and Settings\jarek\Pulpit\Privet\Magisterka\Programy\1\um0427\FWLib\project/RTC.c:284
  1a:	fb93 f1f2 	sdiv	r1, r3, r2
C:\Documents and Settings\jarek\Pulpit\Privet\Magisterka\Programy\1\um0427\FWLib\project/RTC.c:285
  1e:	fb91 f3f7 	sdiv	r3, r1, r7
  22:	425b      	negs	r3, r3
  24:	f240 166d 	movw	r6, #365	; 0x16d
  28:	fb01 3316 	mls	r3, r1, r6, r3
  2c:	f44f 7cc8 	mov.w	ip, #400	; 0x190
  30:	181b      	adds	r3, r3, r0
  32:	fb91 f2fc 	sdiv	r2, r1, ip
  36:	2464      	movs	r4, #100
  38:	1a9b      	subs	r3, r3, r2
  3a:	fb91 f2f4 	sdiv	r2, r1, r4
C:\Documents and Settings\jarek\Pulpit\Privet\Magisterka\Programy\1\um0427\FWLib\project/RTC.c:287
  3e:	eb13 0e02 	adds.w	lr, r3, r2
  42:	d50d      	bpl.n	60 <dtf+0x60>
C:\Documents and Settings\jarek\Pulpit\Privet\Magisterka\Programy\1\um0427\FWLib\project/RTC.c:288
  44:	3901      	subs	r1, #1
C:\Documents and Settings\jarek\Pulpit\Privet\Magisterka\Programy\1\um0427\FWLib\project/RTC.c:289
  46:	fb91 f3f7 	sdiv	r3, r1, r7
  4a:	425b      	negs	r3, r3
  4c:	fb01 3316 	mls	r3, r1, r6, r3
  50:	fb91 f2fc 	sdiv	r2, r1, ip
  54:	181b      	adds	r3, r3, r0
  56:	1a9b      	subs	r3, r3, r2
  58:	fb91 f2f4 	sdiv	r2, r1, r4
  5c:	eb03 0e02 	add.w	lr, r3, r2
C:\Documents and Settings\jarek\Pulpit\Privet\Magisterka\Programy\1\um0427\FWLib\project/RTC.c:292
  60:	fb0e f204 	mul.w	r2, lr, r4
  64:	f640 33f4 	movw	r3, #3060	; 0xbf4
  68:	3234      	adds	r2, #52
  6a:	fb92 f2f3 	sdiv	r2, r2, r3
C:\Documents and Settings\jarek\Pulpit\Privet\Magisterka\Programy\1\um0427\FWLib\project/RTC.c:293
  6e:	1c94      	adds	r4, r2, #2
C:\Documents and Settings\jarek\Pulpit\Privet\Magisterka\Programy\1\um0427\FWLib\project/RTC.c:297
  70:	230c      	movs	r3, #12
  72:	fb94 f0f3 	sdiv	r0, r4, r3
C:\Documents and Settings\jarek\Pulpit\Privet\Magisterka\Programy\1\um0427\FWLib\project/RTC.c:298
  76:	fb00 4313 	mls	r3, r0, r3, r4
  7a:	3301      	adds	r3, #1
  7c:	612b      	str	r3, [r5, #16]
C:\Documents and Settings\jarek\Pulpit\Privet\Magisterka\Programy\1\um0427\FWLib\project/RTC.c:299
  7e:	f44f 7399 	mov.w	r3, #306	; 0x132
  82:	fb02 f203 	mul.w	r2, r2, r3
C:\Documents and Settings\jarek\Pulpit\Privet\Magisterka\Programy\1\um0427\FWLib\project/RTC.c:297
  86:	f501 61fa 	add.w	r1, r1, #2000	; 0x7d0
  8a:	1809      	adds	r1, r1, r0
C:\Documents and Settings\jarek\Pulpit\Privet\Magisterka\Programy\1\um0427\FWLib\project/RTC.c:299
  8c:	3205      	adds	r2, #5
  8e:	f5a3 7394 	sub.w	r3, r3, #296	; 0x128
C:\Documents and Settings\jarek\Pulpit\Privet\Magisterka\Programy\1\um0427\FWLib\project/RTC.c:297
  92:	6169      	str	r1, [r5, #20]
C:\Documents and Settings\jarek\Pulpit\Privet\Magisterka\Programy\1\um0427\FWLib\project/RTC.c:299
  94:	fb92 f2f3 	sdiv	r2, r2, r3
  98:	f10e 0101 	add.w	r1, lr, #1	; 0x1
  9c:	1a89      	subs	r1, r1, r2
  9e:	60e9      	str	r1, [r5, #12]
C:\Documents and Settings\jarek\Pulpit\Privet\Magisterka\Programy\1\um0427\FWLib\project/RTC.c:300
  a0:	bdf0      	pop	{r4, r5, r6, r7, pc}
  a2:	46c0      	nop			(mov r8, r8)
  a4:	0037bb49 	.word	0x0037bb49
Disassembly of section .text.RTC_Save:

00000000 <RTC_Save>:
RTC_Save():
C:\Documents and Settings\jarek\Pulpit\Privet\Magisterka\Programy\1\um0427\FWLib\project/RTC.c:184
   0:	e92d 41f0 	stmdb	sp!, {r4, r5, r6, r7, r8, lr}
   4:	b086      	sub	sp, #24
   6:	4604      	mov	r4, r0
   8:	4688      	mov	r8, r1
C:\Documents and Settings\jarek\Pulpit\Privet\Magisterka\Programy\1\um0427\FWLib\project/RTC.c:188
   a:	f7ff fffe 	bl	0 <RTC_Save>
   e:	4669      	mov	r1, sp
  10:	f7ff fffe 	bl	0 <RTC_Save>
C:\Documents and Settings\jarek\Pulpit\Privet\Magisterka\Programy\1\um0427\FWLib\project/RTC.c:189
  14:	9905      	ldr	r1, [sp, #20]
  16:	6963      	ldr	r3, [r4, #20]
  18:	4299      	cmp	r1, r3
  1a:	d138      	bne.n	8e <RTC_Save+0x8e>
  1c:	6922      	ldr	r2, [r4, #16]
  1e:	9b04      	ldr	r3, [sp, #16]
  20:	4293      	cmp	r3, r2
  22:	d134      	bne.n	8e <RTC_Save+0x8e>
  24:	68e2      	ldr	r2, [r4, #12]
  26:	9b03      	ldr	r3, [sp, #12]
  28:	4293      	cmp	r3, r2
  2a:	d130      	bne.n	8e <RTC_Save+0x8e>
C:\Documents and Settings\jarek\Pulpit\Privet\Magisterka\Programy\1\um0427\FWLib\project/RTC.c:194
  2c:	f5b1 6ffa 	cmp.w	r1, #2000	; 0x7d0
  30:	dd2d      	ble.n	8e <RTC_Save+0x8e>
C:\Documents and Settings\jarek\Pulpit\Privet\Magisterka\Programy\1\um0427\FWLib\project/RTC.c:197
  32:	f640 0349 	movw	r3, #2121	; 0x849
  36:	4299      	cmp	r1, r3
  38:	dc29      	bgt.n	8e <RTC_Save+0x8e>
C:\Documents and Settings\jarek\Pulpit\Privet\Magisterka\Programy\1\um0427\FWLib\project/RTC.c:201
  3a:	68a7      	ldr	r7, [r4, #8]
  3c:	2f17      	cmp	r7, #23
  3e:	dc26      	bgt.n	8e <RTC_Save+0x8e>
C:\Documents and Settings\jarek\Pulpit\Privet\Magisterka\Programy\1\um0427\FWLib\project/RTC.c:204
  40:	6866      	ldr	r6, [r4, #4]
  42:	2e3b      	cmp	r6, #59
  44:	dc23      	bgt.n	8e <RTC_Save+0x8e>
C:\Documents and Settings\jarek\Pulpit\Privet\Magisterka\Programy\1\um0427\FWLib\project/RTC.c:207
  46:	6825      	ldr	r5, [r4, #0]
  48:	2d3b      	cmp	r5, #59
  4a:	dc20      	bgt.n	8e <RTC_Save+0x8e>
C:\Documents and Settings\jarek\Pulpit\Privet\Magisterka\Programy\1\um0427\FWLib\project/RTC.c:211
  4c:	4620      	mov	r0, r4
  4e:	f7ff fffe 	bl	0 <RTC_Save>
C:\Documents and Settings\jarek\Pulpit\Privet\Magisterka\Programy\1\um0427\FWLib\project/RTC.c:213
  52:	233c      	movs	r3, #60
  54:	fb06 f303 	mul.w	r3, r6, r3
  58:	f44f 6261 	mov.w	r2, #3600	; 0xe10
  5c:	fb07 3202 	mla	r2, r7, r2, r3
  60:	4b0d      	ldr	r3, [pc, #52]	(98 <RTC_Save+0x98>)
  62:	1952      	adds	r2, r2, r5
C:\Documents and Settings\jarek\Pulpit\Privet\Magisterka\Programy\1\um0427\FWLib\project/RTC.c:214
  64:	f1b8 0f01 	cmp.w	r8, #1	; 0x1
C:\Documents and Settings\jarek\Pulpit\Privet\Magisterka\Programy\1\um0427\FWLib\project/RTC.c:213
  68:	fb00 2203 	mla	r2, r0, r3, r2
C:\Documents and Settings\jarek\Pulpit\Privet\Magisterka\Programy\1\um0427\FWLib\project/RTC.c:214
  6c:	d007      	beq.n	7e <RTC_Save+0x7e>
  6e:	d303      	bcc.n	78 <RTC_Save+0x78>
  70:	f1b8 0f02 	cmp.w	r8, #2	; 0x2
  74:	d007      	beq.n	86 <RTC_Save+0x86>
  76:	e008      	b.n	8a <RTC_Save+0x8a>
C:\Documents and Settings\jarek\Pulpit\Privet\Magisterka\Programy\1\um0427\FWLib\project/RTC.c:216
  78:	4b08      	ldr	r3, [pc, #32]	(9c <RTC_Save+0x9c>)
  7a:	601a      	str	r2, [r3, #0]
  7c:	e005      	b.n	8a <RTC_Save+0x8a>
C:\Documents and Settings\jarek\Pulpit\Privet\Magisterka\Programy\1\um0427\FWLib\project/RTC.c:219
  7e:	4b07      	ldr	r3, [pc, #28]	(9c <RTC_Save+0x9c>)
  80:	4640      	mov	r0, r8
  82:	605a      	str	r2, [r3, #4]
C:\Documents and Settings\jarek\Pulpit\Privet\Magisterka\Programy\1\um0427\FWLib\project/RTC.c:220
  84:	e004      	b.n	90 <RTC_Save+0x90>
C:\Documents and Settings\jarek\Pulpit\Privet\Magisterka\Programy\1\um0427\FWLib\project/RTC.c:222
  86:	4b05      	ldr	r3, [pc, #20]	(9c <RTC_Save+0x9c>)
  88:	609a      	str	r2, [r3, #8]
  8a:	2001      	movs	r0, #1
  8c:	e000      	b.n	90 <RTC_Save+0x90>
  8e:	2000      	movs	r0, #0
C:\Documents and Settings\jarek\Pulpit\Privet\Magisterka\Programy\1\um0427\FWLib\project/RTC.c:226
  90:	b006      	add	sp, #24
  92:	e8bd 81f0 	ldmia.w	sp!, {r4, r5, r6, r7, r8, pc}
  96:	46c0      	nop			(mov r8, r8)
  98:	00015180 	.word	0x00015180
  9c:	00000000 	.word	0x00000000
Disassembly of section .text.RTC_Read:

00000000 <RTC_Read>:
RTC_Read():
C:\Documents and Settings\jarek\Pulpit\Privet\Magisterka\Programy\1\um0427\FWLib\project/RTC.c:90
   0:	4b16      	ldr	r3, [pc, #88]	(5c <RTC_Read+0x5c>)
C:\Documents and Settings\jarek\Pulpit\Privet\Magisterka\Programy\1\um0427\FWLib\project/RTC.c:87
   2:	b570      	push	{r4, r5, r6, lr}
   4:	4605      	mov	r5, r0
C:\Documents and Settings\jarek\Pulpit\Privet\Magisterka\Programy\1\um0427\FWLib\project/RTC.c:90
   6:	2000      	movs	r0, #0
C:\Documents and Settings\jarek\Pulpit\Privet\Magisterka\Programy\1\um0427\FWLib\project/RTC.c:92
   8:	2901      	cmp	r1, #1
C:\Documents and Settings\jarek\Pulpit\Privet\Magisterka\Programy\1\um0427\FWLib\project/RTC.c:90
   a:	60d8      	str	r0, [r3, #12]
C:\Documents and Settings\jarek\Pulpit\Privet\Magisterka\Programy\1\um0427\FWLib\project/RTC.c:92
   c:	d007      	beq.n	1e <RTC_Read+0x1e>
   e:	d303      	bcc.n	18 <RTC_Read+0x18>
  10:	2902      	cmp	r1, #2
  12:	d007      	beq.n	24 <RTC_Read+0x24>
  14:	4604      	mov	r4, r0
  16:	e007      	b.n	28 <RTC_Read+0x28>
C:\Documents and Settings\jarek\Pulpit\Privet\Magisterka\Programy\1\um0427\FWLib\project/RTC.c:94
  18:	4b11      	ldr	r3, [pc, #68]	(60 <RTC_Read+0x60>)
  1a:	681c      	ldr	r4, [r3, #0]
C:\Documents and Settings\jarek\Pulpit\Privet\Magisterka\Programy\1\um0427\FWLib\project/RTC.c:95
  1c:	e004      	b.n	28 <RTC_Read+0x28>
C:\Documents and Settings\jarek\Pulpit\Privet\Magisterka\Programy\1\um0427\FWLib\project/RTC.c:97
  1e:	4b10      	ldr	r3, [pc, #64]	(60 <RTC_Read+0x60>)
  20:	685c      	ldr	r4, [r3, #4]
C:\Documents and Settings\jarek\Pulpit\Privet\Magisterka\Programy\1\um0427\FWLib\project/RTC.c:98
  22:	e001      	b.n	28 <RTC_Read+0x28>
C:\Documents and Settings\jarek\Pulpit\Privet\Magisterka\Programy\1\um0427\FWLib\project/RTC.c:100
  24:	4b0e      	ldr	r3, [pc, #56]	(60 <RTC_Read+0x60>)
  26:	689c      	ldr	r4, [r3, #8]
C:\Documents and Settings\jarek\Pulpit\Privet\Magisterka\Programy\1\um0427\FWLib\project/RTC.c:105
  28:	f44f 6061 	mov.w	r0, #3600	; 0xe10
  2c:	fbb4 f1f0 	udiv	r1, r4, r0
  30:	2318      	movs	r3, #24
  32:	fbb1 f2f3 	udiv	r2, r1, r3
  36:	fb02 1313 	mls	r3, r2, r3, r1
C:\Documents and Settings\jarek\Pulpit\Privet\Magisterka\Programy\1\um0427\FWLib\project/RTC.c:107
  3a:	fb01 4010 	mls	r0, r1, r0, r4
C:\Documents and Settings\jarek\Pulpit\Privet\Magisterka\Programy\1\um0427\FWLib\project/RTC.c:105
  3e:	60ab      	str	r3, [r5, #8]
C:\Documents and Settings\jarek\Pulpit\Privet\Magisterka\Programy\1\um0427\FWLib\project/RTC.c:107
  40:	233c      	movs	r3, #60
  42:	fbb0 f2f3 	udiv	r2, r0, r3
C:\Documents and Settings\jarek\Pulpit\Privet\Magisterka\Programy\1\um0427\FWLib\project/RTC.c:109
  46:	fb02 0313 	mls	r3, r2, r3, r0
C:\Documents and Settings\jarek\Pulpit\Privet\Magisterka\Programy\1\um0427\FWLib\project/RTC.c:113
  4a:	4806      	ldr	r0, [pc, #24]	(64 <RTC_Read+0x64>)
C:\Documents and Settings\jarek\Pulpit\Privet\Magisterka\Programy\1\um0427\FWLib\project/RTC.c:107
  4c:	606a      	str	r2, [r5, #4]
C:\Documents and Settings\jarek\Pulpit\Privet\Magisterka\Programy\1\um0427\FWLib\project/RTC.c:109
  4e:	602b      	str	r3, [r5, #0]
C:\Documents and Settings\jarek\Pulpit\Privet\Magisterka\Programy\1\um0427\FWLib\project/RTC.c:113
  50:	fbb4 f0f0 	udiv	r0, r4, r0
  54:	4629      	mov	r1, r5
  56:	f7ff fffe 	bl	0 <RTC_Read>
C:\Documents and Settings\jarek\Pulpit\Privet\Magisterka\Programy\1\um0427\FWLib\project/RTC.c:114
  5a:	bd70      	pop	{r4, r5, r6, pc}
	...
  64:	00015180 	.word	0x00015180
Disassembly of section .text.RTC_SaveTime:

00000000 <RTC_SaveTime>:
RTC_SaveTime():
C:\Documents and Settings\jarek\Pulpit\Privet\Magisterka\Programy\1\um0427\FWLib\project/RTC.c:152
   0:	b570      	push	{r4, r5, r6, lr}
C:\Documents and Settings\jarek\Pulpit\Privet\Magisterka\Programy\1\um0427\FWLib\project/RTC.c:156
   2:	6883      	ldr	r3, [r0, #8]
C:\Documents and Settings\jarek\Pulpit\Privet\Magisterka\Programy\1\um0427\FWLib\project/RTC.c:152
   4:	b086      	sub	sp, #24
C:\Documents and Settings\jarek\Pulpit\Privet\Magisterka\Programy\1\um0427\FWLib\project/RTC.c:156
   6:	2b17      	cmp	r3, #23
C:\Documents and Settings\jarek\Pulpit\Privet\Magisterka\Programy\1\um0427\FWLib\project/RTC.c:152
   8:	4605      	mov	r5, r0
   a:	460e      	mov	r6, r1
C:\Documents and Settings\jarek\Pulpit\Privet\Magisterka\Programy\1\um0427\FWLib\project/RTC.c:156
   c:	dc2b      	bgt.n	66 <RTC_SaveTime+0x66>
C:\Documents and Settings\jarek\Pulpit\Privet\Magisterka\Programy\1\um0427\FWLib\project/RTC.c:159
   e:	6843      	ldr	r3, [r0, #4]
  10:	2b3b      	cmp	r3, #59
  12:	dc28      	bgt.n	66 <RTC_SaveTime+0x66>
C:\Documents and Settings\jarek\Pulpit\Privet\Magisterka\Programy\1\um0427\FWLib\project/RTC.c:162
  14:	6803      	ldr	r3, [r0, #0]
  16:	2b3b      	cmp	r3, #59
  18:	dc25      	bgt.n	66 <RTC_SaveTime+0x66>
C:\Documents and Settings\jarek\Pulpit\Privet\Magisterka\Programy\1\um0427\FWLib\project/RTC.c:165
  1a:	4668      	mov	r0, sp
  1c:	f7ff fffe 	bl	0 <RTC_SaveTime>
C:\Documents and Settings\jarek\Pulpit\Privet\Magisterka\Programy\1\um0427\FWLib\project/RTC.c:166
  20:	4668      	mov	r0, sp
  22:	f7ff fffe 	bl	0 <RTC_SaveTime>
C:\Documents and Settings\jarek\Pulpit\Privet\Magisterka\Programy\1\um0427\FWLib\project/RTC.c:168
  26:	686a      	ldr	r2, [r5, #4]
  28:	233c      	movs	r3, #60
  2a:	fb02 f203 	mul.w	r2, r2, r3
  2e:	68a9      	ldr	r1, [r5, #8]
  30:	f44f 6361 	mov.w	r3, #3600	; 0xe10
  34:	fb01 2303 	mla	r3, r1, r3, r2
  38:	682a      	ldr	r2, [r5, #0]
C:\Documents and Settings\jarek\Pulpit\Privet\Magisterka\Programy\1\um0427\FWLib\project/RTC.c:165
  3a:	466c      	mov	r4, sp
C:\Documents and Settings\jarek\Pulpit\Privet\Magisterka\Programy\1\um0427\FWLib\project/RTC.c:168
  3c:	189b      	adds	r3, r3, r2
  3e:	4a0b      	ldr	r2, [pc, #44]	(6c <RTC_SaveTime+0x6c>)
C:\Documents and Settings\jarek\Pulpit\Privet\Magisterka\Programy\1\um0427\FWLib\project/RTC.c:169
  40:	2e01      	cmp	r6, #1
C:\Documents and Settings\jarek\Pulpit\Privet\Magisterka\Programy\1\um0427\FWLib\project/RTC.c:168
  42:	fb00 3002 	mla	r0, r0, r2, r3
C:\Documents and Settings\jarek\Pulpit\Privet\Magisterka\Programy\1\um0427\FWLib\project/RTC.c:169
  46:	d006      	beq.n	56 <RTC_SaveTime+0x56>
  48:	d302      	bcc.n	50 <RTC_SaveTime+0x50>
  4a:	2e02      	cmp	r6, #2
  4c:	d007      	beq.n	5e <RTC_SaveTime+0x5e>
  4e:	e008      	b.n	62 <RTC_SaveTime+0x62>
C:\Documents and Settings\jarek\Pulpit\Privet\Magisterka\Programy\1\um0427\FWLib\project/RTC.c:171
  50:	4b07      	ldr	r3, [pc, #28]	(70 <RTC_SaveTime+0x70>)
  52:	6018      	str	r0, [r3, #0]
  54:	e005      	b.n	62 <RTC_SaveTime+0x62>
C:\Documents and Settings\jarek\Pulpit\Privet\Magisterka\Programy\1\um0427\FWLib\project/RTC.c:174
  56:	4b06      	ldr	r3, [pc, #24]	(70 <RTC_SaveTime+0x70>)
  58:	6058      	str	r0, [r3, #4]
  5a:	4630      	mov	r0, r6
C:\Documents and Settings\jarek\Pulpit\Privet\Magisterka\Programy\1\um0427\FWLib\project/RTC.c:175
  5c:	e004      	b.n	68 <RTC_SaveTime+0x68>
C:\Documents and Settings\jarek\Pulpit\Privet\Magisterka\Programy\1\um0427\FWLib\project/RTC.c:177
  5e:	4b04      	ldr	r3, [pc, #16]	(70 <RTC_SaveTime+0x70>)
  60:	6098      	str	r0, [r3, #8]
  62:	2001      	movs	r0, #1
  64:	e000      	b.n	68 <RTC_SaveTime+0x68>
  66:	2000      	movs	r0, #0
C:\Documents and Settings\jarek\Pulpit\Privet\Magisterka\Programy\1\um0427\FWLib\project/RTC.c:181
  68:	b006      	add	sp, #24
  6a:	bd70      	pop	{r4, r5, r6, pc}
  6c:	00015180 	.word	0x00015180
  70:	00000000 	.word	0x00000000
Disassembly of section .text.RTC_SaveDate:

00000000 <RTC_SaveDate>:
RTC_SaveDate():
C:\Documents and Settings\jarek\Pulpit\Privet\Magisterka\Programy\1\um0427\FWLib\project/RTC.c:116
   0:	b570      	push	{r4, r5, r6, lr}
   2:	b086      	sub	sp, #24
   4:	4604      	mov	r4, r0
   6:	460d      	mov	r5, r1
C:\Documents and Settings\jarek\Pulpit\Privet\Magisterka\Programy\1\um0427\FWLib\project/RTC.c:121
   8:	f7ff fffe 	bl	0 <RTC_SaveDate>
   c:	4669      	mov	r1, sp
   e:	f7ff fffe 	bl	0 <RTC_SaveDate>
C:\Documents and Settings\jarek\Pulpit\Privet\Magisterka\Programy\1\um0427\FWLib\project/RTC.c:122
  12:	9905      	ldr	r1, [sp, #20]
  14:	6963      	ldr	r3, [r4, #20]
C:\Documents and Settings\jarek\Pulpit\Privet\Magisterka\Programy\1\um0427\FWLib\project/RTC.c:121
  16:	466e      	mov	r6, sp
C:\Documents and Settings\jarek\Pulpit\Privet\Magisterka\Programy\1\um0427\FWLib\project/RTC.c:122
  18:	4299      	cmp	r1, r3
  1a:	d134      	bne.n	86 <RTC_SaveDate+0x86>
  1c:	6922      	ldr	r2, [r4, #16]
  1e:	9b04      	ldr	r3, [sp, #16]
  20:	4293      	cmp	r3, r2
  22:	d130      	bne.n	86 <RTC_SaveDate+0x86>
  24:	68e2      	ldr	r2, [r4, #12]
  26:	9b03      	ldr	r3, [sp, #12]
  28:	4293      	cmp	r3, r2
  2a:	d12c      	bne.n	86 <RTC_SaveDate+0x86>
C:\Documents and Settings\jarek\Pulpit\Privet\Magisterka\Programy\1\um0427\FWLib\project/RTC.c:127
  2c:	f5b1 6ffa 	cmp.w	r1, #2000	; 0x7d0
  30:	dd29      	ble.n	86 <RTC_SaveDate+0x86>
C:\Documents and Settings\jarek\Pulpit\Privet\Magisterka\Programy\1\um0427\FWLib\project/RTC.c:130
  32:	f640 0349 	movw	r3, #2121	; 0x849
  36:	4299      	cmp	r1, r3
  38:	dc25      	bgt.n	86 <RTC_SaveDate+0x86>
C:\Documents and Settings\jarek\Pulpit\Privet\Magisterka\Programy\1\um0427\FWLib\project/RTC.c:133
  3a:	4629      	mov	r1, r5
  3c:	4668      	mov	r0, sp
  3e:	f7ff fffe 	bl	0 <RTC_SaveDate>
C:\Documents and Settings\jarek\Pulpit\Privet\Magisterka\Programy\1\um0427\FWLib\project/RTC.c:135
  42:	4620      	mov	r0, r4
  44:	f7ff fffe 	bl	0 <RTC_SaveDate>
C:\Documents and Settings\jarek\Pulpit\Privet\Magisterka\Programy\1\um0427\FWLib\project/RTC.c:137
  48:	9a01      	ldr	r2, [sp, #4]
  4a:	233c      	movs	r3, #60
  4c:	fb02 f203 	mul.w	r2, r2, r3
  50:	9902      	ldr	r1, [sp, #8]
  52:	f44f 6361 	mov.w	r3, #3600	; 0xe10
  56:	fb01 2303 	mla	r3, r1, r3, r2
  5a:	9a00      	ldr	r2, [sp, #0]
  5c:	189b      	adds	r3, r3, r2
  5e:	4a0b      	ldr	r2, [pc, #44]	(8c <RTC_SaveDate+0x8c>)
C:\Documents and Settings\jarek\Pulpit\Privet\Magisterka\Programy\1\um0427\FWLib\project/RTC.c:138
  60:	2d01      	cmp	r5, #1
C:\Documents and Settings\jarek\Pulpit\Privet\Magisterka\Programy\1\um0427\FWLib\project/RTC.c:137
  62:	fb00 3202 	mla	r2, r0, r2, r3
C:\Documents and Settings\jarek\Pulpit\Privet\Magisterka\Programy\1\um0427\FWLib\project/RTC.c:138
  66:	d006      	beq.n	76 <RTC_SaveDate+0x76>
  68:	d302      	bcc.n	70 <RTC_SaveDate+0x70>
  6a:	2d02      	cmp	r5, #2
  6c:	d007      	beq.n	7e <RTC_SaveDate+0x7e>
  6e:	e008      	b.n	82 <RTC_SaveDate+0x82>
C:\Documents and Settings\jarek\Pulpit\Privet\Magisterka\Programy\1\um0427\FWLib\project/RTC.c:140
  70:	4b07      	ldr	r3, [pc, #28]	(90 <RTC_SaveDate+0x90>)
  72:	601a      	str	r2, [r3, #0]
  74:	e005      	b.n	82 <RTC_SaveDate+0x82>
C:\Documents and Settings\jarek\Pulpit\Privet\Magisterka\Programy\1\um0427\FWLib\project/RTC.c:143
  76:	4b06      	ldr	r3, [pc, #24]	(90 <RTC_SaveDate+0x90>)
  78:	4628      	mov	r0, r5
  7a:	605a      	str	r2, [r3, #4]
C:\Documents and Settings\jarek\Pulpit\Privet\Magisterka\Programy\1\um0427\FWLib\project/RTC.c:144
  7c:	e004      	b.n	88 <RTC_SaveDate+0x88>
C:\Documents and Settings\jarek\Pulpit\Privet\Magisterka\Programy\1\um0427\FWLib\project/RTC.c:146
  7e:	4b04      	ldr	r3, [pc, #16]	(90 <RTC_SaveDate+0x90>)
  80:	609a      	str	r2, [r3, #8]
  82:	2001      	movs	r0, #1
  84:	e000      	b.n	88 <RTC_SaveDate+0x88>
  86:	2000      	movs	r0, #0
C:\Documents and Settings\jarek\Pulpit\Privet\Magisterka\Programy\1\um0427\FWLib\project/RTC.c:150
  88:	b006      	add	sp, #24
  8a:	bd70      	pop	{r4, r5, r6, pc}
  8c:	00015180 	.word	0x00015180
  90:	00000000 	.word	0x00000000
